:107800000C94343C0C94513C0C94513C0C94513CE1
:107810000C94513C0C94513C0C94513C0C94513CB4
:107820000C94513C0C94513C0C94513C0C94513CA4
:107830000C94513C0C94513C0C94513C0C94513C94
:107840000C94513C0C94513C0C94513C0C94513C84
:107850000C94513C0C94513C0C94513C0C94513C74
:107860000C94513C0C94513C11241FBECFEFD8E036
:10787000DEBFCDBF11E0A0E0B1E0ECECFDE702C05F
:1078800005900D92A230B107D9F722E0A2E0B1E055
:1078900001C01D92AD30B207E1F70E940A3D0C9481
:1078A000E43E0C94003C9091C00095FFFCCF809387
:1078B000C6000895CF93982F8595859585958595D4
:1078C000805D9F709A3014F0C7E501C0C0E3C90F16
:1078D0000E94533C8C2FCF910C94533CCF92DF925B
:1078E000EF92FF92C12CD12C76018091C00087FDD0
:1078F00013C08FEFC81AD80AE80AF80A81E2C8163E
:1079000081EAD80687E0E806F10478F3E091020105
:10791000F09103010995E9CF8091C600FF90EF90A7
:10792000DF90CF900895CF930E946E3CC82F0E94A5
:10793000533CC13614F089EA03C0C0331CF080ED1B
:107940008C0F01C08C2FCF910895CF930E94933C50
:10795000C82F0E94933C90E1C99F800D1124CF91C4
:107960000895CF93C82FCC2321F00E946E3CC150C4
:10797000FACFCF910895CF93C82F0E946E3C8032EA
:1079800051F484E10E94533C8C2F0E94533C80E1CF
:10799000CF910C94533C809104018F5F809304013C
:1079A000853031F4E0910201F0910301CF91099407
:1079B000CF9108950E946E3C803231F484E10E94A0
:1079C000533C80E10C94533C809104018F5F809381
:1079D0000401853029F4E0910201F091030109943A
:1079E00008958823B1F02D9A2FEF30E792E02150CF
:1079F00030409040E1F700C000002D982FEF30E7B5
:107A000092E0215030409040E1F700C000008150EA
:107A1000E8CF08950000E0E0F0E0E49182E0809398
:107A2000C00080E18093C4001092C50088E180937B
:107A3000C10086E08093C2005098589A259A81E050
:107A40000E94F13CFF24F3940E946E3C803309F4C1
:107A500042C08133E1F40E946E3C803209F0A6C13D
:107A600084E10E94533C81E40E94533C86E50E94DD
:107A7000533C82E50E94533C80E20E94533C89E4DF
:107A80000E94533C83E50E94533C80E586C18034CC
:107A900039F40E946E3C8638F0F00E946E3C1BC0A8
:107AA0008134A1F40E946E3C803811F482E003C05E
:107AB000813821F481E00E94BB3CC6CF823811F4AA
:107AC00080E1F9CF8839C9F583E0F5CF823431F40C
:107AD00084E10E94B13C0E94DA3CB6CF853411F4B7
:107AE00085E0F7CF982F9D7F9035A9F3813599F3E5
:107AF000853549F40E946E3C809306010E946E3CDD
:107B000080930701E8CF8635D1F40E946E3C803324
:107B100089F40E946E3C0E946E3C182F0E946E3CBD
:107B2000111102C08EE1C7CF113011F485E9C3CF26
:107B30008FE0C1CF83E00E94B13C80E0BCCF8436AF
:107B400009F0C6C00E946E3C809309020E946E3C00
:107B50008093080280910C028E7F80930C020E9419
:107B60006E3C853429F480910C02816080930C0274
:107B700008E011E02091080230910902C801885004
:107B800091408217930730F40E946E3CF801819374
:107B90008F01F0CF0E946E3C803209F007C18091C6
:107BA0000C02209106013091070180FF29C0220FAD
:107BB000331F3093070120930601E8E0F1E02091A4
:107BC000080230910902CF01885091408217930733
:107BD00008F07CC0F999FECF8091060190910701D1
:107BE00092BD81BD819180BDFA9AF99A809106017A
:107BF0009091070101969093070180930601DFCFD2
:107C000080910701880F880B8F2180930B02220F30
:107C1000331F30930701209306018091080280FFF3
:107C200009C080910802909109020196909309027F
:107C300080930802F894F999FECF1127E09106018C
:107C4000F0910701C8E0D1E080910802909109020B
:107C5000103091F40091570001700130D9F303E026
:107C600000935700E8950091570001700130D9F357
:107C700001E100935700E895099019900091570091
:107C800001700130D9F301E000935700E895139596
:107C9000103498F011270091570001700130D9F38A
:107CA00005E000935700E8950091570001700130FE
:107CB000D9F301E100935700E8953296029709F055
:107CC000C7CF103011F00296E5CF112484E165C0D2
:107CD000843709F052C00E946E3C809309020E94D2
:107CE0006E3C809308028091060190910701880FF5
:107CF000991F90930701809306010E946E3C90911A
:107D00000C02853411F4916001C09E7F90930C02A7
:107D10000E946E3C803209F097CE84E10E94533C71
:107D200000E010E0809108029091090208171907FD
:107D3000B0F580910C0280FF0BC0F999FECF8091C5
:107D400006019091070192BD81BDF89A80B507C0E8
:107D500081FD07C0E0910601F091070184910E9426
:107D6000533C809106019091070101969093070181
:107D7000809306010F5F1F4FD5CF8537A1F40E9476
:107D80006E3C803299F484E10E94533C8EE10E9463
:107D9000533C85E90E94533C8FE00E94533C80E1B4
:107DA0000E94533C51CE863709F4C7CE809104011E
:107DB0008F5F80930401853009F046CEE091020187
:0C7DC000F0910301099540CEF894FFCF2C
:027DCC00800035
:040000030000780081
:00000001FF
